:100000001BC1000043C1000041C100003FC100000E
:100010003DC100003BC1000039C1000037C10000F4
:1000200035C1000033C1000035C400002FC10000FD
:100030002DC100002BC1000029C1000027C1000014
:1000400025C1000023C1000021C100001FC1000024
:100050001DC100001BC1000019C1000017C1000034
:1000600015C1000013C1000011C100000FC1000044
:100070000DC100000BC1000009C1000007C1000054
:1000800005C1000003C1000001C10000FFC0000065
:10009000FDC00000FBC00000120100020000004093
:1000A00000000000001001020301090252000301D8
:1000B00000C03209040000010300020009211101FF
:1000C000000122340007058103080006090401002D
:1000D0000103000101092111010001223B00070574
:1000E00082030800140904020002080650020705F2
:1000F0008302400000070504024000000C034F008B
:1001000054004C004C0043002603430068006F007D
:1001100072006400690074006500200050007200E5
:100120006F0074006F0074007900700065001C039C
:10013000300030003000300030003000300030003F
:1001400030003000300030003000040309040501A5
:100150000902A1010901A1000509190129031500DE
:100160002501750195038102750595018101050140
:100170000930093109381581257F750895038106F5
:10018000C0C005010906A101050719E029E715000E
:100190002501750195088102810119002965150065
:1001A00025657508950681000508190129051500C2
:1001B000250175019505910295039101C0002C2A36
:1001C000E1080C11061712160915101A14040B0772
:1001D0001C0F13050D180A191B0E1D002B36373383
:1001E000342F3031381E1F20212223242526272D8D
:1001F0002E2835E2E0504F52514B4E494C4A4D4665
:1002000048E539E3E73A3B3C3D3E3F404142434409
:1002100045292941544D454C202020415439305521
:100220005342313238204D20532020302E303000C0
:100230008003021F0000000011241FBECFEFD0E298
:10024000DEBFCDBF80E090E020E80FB6F8942093A9
:100250006100809361000FBE81E011E0A0E0B1E099
:10026000ECE3FDE200E00BBF02C007900D92A4306A
:10027000B107D9F711E0A4E0B1E001C01D92AF349D
:10028000B107E1F70E948B160C949C16B9CE8FB77C
:10029000F89497EF94BF98E10FB6F89490936000AC
:1002A000109260000FBE87FF01C078940895C7D3F5
:1002B000F6D60E94A9090E94EB0AF9CFC2D356D6FE
:1002C000E4D70C94F90AFADFF2CF9091EB00916039
:1002D0009093EB008093EC008091ED008270862B70
:1002E0008093ED008091ED0082608093ED0080911D
:1002F000EE00881F8827881F08958091D8008F7B83
:100300008093D8008091D90081FF21C01092E9002C
:100310008091EB0080FD1BC01092E9008091EB0002
:1003200081608093EB0082E08093EC008091ED008F
:10033000827080638093ED008091ED0082608093F5
:10034000ED008091EE00881F8827881F089580E0C7
:1003500008957894E8EDF0E080818F768083808145
:100360008069808380818F7B8083789408958EE07C
:1003700089BD09B400FEFDCF8091D8008F7D8093A8
:10038000D800BBDF8091E0008E7F8093E0008091F9
:10039000E20081608093E2008091E20088608093B7
:1003A000E20008958091D90080FF14C0809104017B
:1003B000882381F481E08093040110920601D6D550
:1003C00080910701909108018260909308018093C9
:1003D0000701CDDF8091D90080FD13C02FC010929E
:1003E0000401109226018091070190910801846018
:1003F00090930801809307018091D80080628093D8
:10040000D800809107019091080190FF10C0809161
:100410000701909108019E7F909308018093070146
:1004200081E08093EA001092EA0010922601109277
:10043000E9008091E80083FF06C006C080910401B6
:100440008130F9F6CCCF08950F931F93DF93CF93AC
:1004500000D0CDB7DEB78091E8008B7F8093E800B5
:100460001091F1000091F1000630F9F0073068F4C6
:10047000013009F413C1013008F480C1033009F4DC
:1004800041C1053009F0EDC1D2C0093009F4EFC017
:100490000A3020F4083009F0E4C1A4C00A3009F49D
:1004A0009BC10B3009F0DDC1BAC1103809F0D9C1C8
:1004B0006091F1008091F100813019F0823089F46F
:1004C00006C082E18093270188E990E005C082E5BB
:1004D000809327018AEA90E0909329018093280174
:1004E00004C0D2D2882309F4BCC18091F10080916C
:1004F000F1008091F10089838091F1008A838091DD
:10050000E800877F8093E80029813A818091270164
:1005100090E08217930730F48F739070892B21F449
:1005200061E003C02093270160E08091E8008F7EA6
:100530008093E80020912801309129014091270102
:1005400022C08091E80084FF03C0F90190E00FC051
:100550008091E80080FFF5CFF8CF542F51509034B0
:1005600049F09F5F84918093F1003196452F9F0160
:10057000442399F78091E80084FD12C08091E8003F
:100580008E7F8093E800442339F420932801309330
:100590002901109227010AC08091E80084FFD8CF7A
:1005A000209328013093290140932701613069F499
:1005B0008091E80084FD09C08091E80080FFFCCFB5
:1005C0008091E8008E7F8093E8008091E80084FFAE
:1005D000FCCF8091E8008F7E8093E8008091E80056
:1005E0008B7F22C0103809F03CC18091E800877FE2
:1005F0008093E800809126018093F1008091E800CB
:100600008E7F8093E8008091E8008F778093E800E8
:100610008091E80082FFFCCF8091E8008B7F80937F
:10062000E8008091E8008F778093E8002CC11123C7
:1006300009F017C19091F1008091E3009F778078D5
:10064000982B9093E3008091E800877F8093E800E7
:100650008091E8008E7F8093E8008091E80080FF21
:10066000FCCF8091E30080688093E3000CC11123EC
:1006700009F0F7C09091F100923008F0F2C080913B
:10068000E800877F8093E800909326018091E8003E
:100690008E7F8093E800892FA4D3F5C01123C1F188
:1006A000123009F0DEC08091F1009091F1008823B2
:1006B00009F0D7C0E091F100EF77E093E900809175
:1006C000EB0080FF43C0EE23B1F08091EB0080612E
:1006D0008093EB0081E090E00E2E02C0880F991FFE
:1006E0000A94E2F78093EA001092EA008091EB000E
:1006F00088608093EB001092E900F0E0E15EFE4F2D
:10070000108233C0112321F0123009F0AAC003C0B7
:100710008091F100A6C08091F1009091F1008823B2
:1007200009F09FC0E091F100EF7751F48091EB0068
:1007300080628093EB008091E800877F8093E800DF
:10074000E093E9008091EB0080FD03C01092E90086
:1007500088C08091EB0080628093EB001092E900EA
:10076000F0E0E15EFE4F81E080838091E800877FCA
:100770008093E8008091E8008E7F56CF8091F10051
:100780008091F100E091F100113829F0123859F010
:10079000103809F066C08091E800877F8093E800F8
:1007A0001092F1000DC08091E800877F8093E800EF
:1007B000F0E0EF77F070E15EFE4F80818093F10012
:1007C0001092F1008091E8008E7F8093E800809184
:1007D000E80082FFFCCF20CF113809F042C08091A1
:1007E000F1008091F1009091F10099839091F100D6
:1007F0009A838823B1F58091E800877F8093E80091
:1008000089819A812AD18093F1008091E8008E7FBE
:100810008093E8008091E80082FFFCCFFDCE11308C
:1008200001F56091F1008091F1009091F1009983C0
:100830009091F1009A838823A1F48091E800877F4A
:100840008093E80089819A810AD11092E900809111
:10085000E8008E7F8093E8008091E80080FFFCCF65
:1008600012C0812F602FDCD2882369F48091EB00C5
:1008700080628093EB008091E800877F8093E8009E
:1008800081E080931F010F900F90CF91DF911F9116
:100890000F9108951F920F920FB60F920BB60F9201
:1008A00011242F933F934F935F936F937F938F9375
:1008B0009F93AF93BF93EF93FF938091E10082FFEB
:1008C00008C08091E20082FF04C08BEF8093E100BA
:1008D0005AD38091E10080FF41C08091E20080FF07
:1008E0003DC0809106018130D9F480912601882392
:1008F000B9F08091E2008E7F8093E2008FEE8093CA
:10090000E1008091E20080618093E20089B58D7FF3
:1009100089BD19BC8091D80080628093D8001DC029
:100920008FEE8093E1008091070190910801806231
:1009300090930801809307018EEF8093E1008091EE
:10094000E20080618093E2008091D8008062809311
:10095000D80089B58D7F89BD19BC1BD38091E1007A
:1009600084FF27C08091E20084FF23C009B400FC0B
:1009700005C08EE089BD09B400FEFDCF8091D8008E
:100980008F7D8093D8008FEE8093E1008091E2000C
:100990008F7E8093E200809107019091080180642E
:1009A00090930801809307018091E2008160809319
:1009B000E2008091E10085FF1AC08091E20085FF8E
:1009C00016C08091E2008F7E8093E2008FED8093CD
:1009D000E1008091E2008F7D8093E2008091070129
:1009E000909108018068909308018093070180919D
:1009F000E10083FF11C08091E20083FF0DC087EF0B
:100A00008093E1007ADC8091070190910801916068
:100A10009093080180930701FF91EF91BF91AF91EF
:100A20009F918F917F916F915F914F913F912F9106
:100A30000F900BBE0F900FBE0F901F901895B2CC69
:100A40000895E7EDF0E080818160808380818F7B75
:100A500080838081806880837CCC80E00895892BAE
:100A600091F481E08093E9008091EB0080618093B4
:100A7000EB0082E08093EA001092EA008091EB00A4
:100A800088608093EB000895833031F5613069F020
:100A9000613028F0623079F06330F1F412C084E004
:100AA000809327018AE491E011C08CE080932701B4
:100AB0008CEF90E00BC086E28093270188E091E004
:100AC00005C08CE1809327018EE291E0909329018B
:100AD0008093280181E0089580E00895DF93CF930B
:100AE00000D000D0CDB7DEB78091F1008B8380912C
:100AF000F1008C838B819C81009719F0019781F420
:100B000006C084E3809327018EE491E005C08BE367
:100B10008093270182E891E0909329018093280136
:100B20008091F10089838091F1008A838091E800AF
:100B3000877F8093E80029813A818091270190E0A6
:100B40008217930770F48F739070892B11F461E012
:100B500001C060E0209128013091290140912701D6
:100B60001CC020932701F5CF8091E80080FFFCCFC7
:100B7000F90190E00AC0542F5150903449F09F5F22
:100B800084918093F1003196452F9F01442399F77A
:100B90008091E8008E7F8093E800442359F0809193
:100BA000E80082FFE1CF2093280130932901409390
:100BB000270106C0209328013093290110922701B4
:100BC0008091E80082FD0FC0613049F48091E80017
:100BD00080FFFCCF8091E8008E7F8093E8008091B9
:100BE000E80082FFFCCF8091E8008B7F8093E800D3
:100BF0008091E8008F778093E8000F900F900F901E
:100C00000F90CF91DF9108958091E800877F8093C6
:100C1000E8008091E8008E7F8093E8008091E800F2
:100C200082FFFCCF8091E8008B7F8093E800809169
:100C3000E8008F778093E8008091E8008E7F8093B2
:100C4000E8000895DF93CF9300D000D0CDB7DEB792
:100C50008091F1008B838091F1008C838091F10071
:100C600089838091F1008A838091E800877F809357
:100C7000E80089819A81892B49F08091090180934C
:100C8000F1008091E8008E7F8093E8008091E80079
:100C900082FFFCCF8091E8008B7F8093E8008091F9
:100CA000E8008F778093E8000F900F900F900F90DF
:100CB000CF91DF910895DF93CF9300D000D0CDB7CF
:100CC000DEB78091F1008B838091F1008C838B8162
:100CD0009C81009719F0019781F406C089E0809308
:100CE00027018CEB90E005C089E08093270185ED1A
:100CF00090E090932901809328018091F1008983ED
:100D00008091F1008A838091E800877F8093E800DA
:100D100029813A818091270190E08217930770F42E
:100D20008F739070892B11F461E001C060E0209115
:100D3000280130912901409127011CC020932701EF
:100D4000F5CF8091E80080FFFCCFF90190E00AC068
:100D5000542F5150903449F09F5F84918093F1005B
:100D60003196452F9F01442399F78091E8008E7FAB
:100D70008093E800442359F08091E80082FFE1CF9E
:100D800020932801309329014093270106C0209326
:100D9000280130932901109227018091E80082FDFB
:100DA0000FC0613049F48091E80080FFFCCF809152
:100DB000E8008E7F8093E8008091E80082FFFCCFFE
:100DC0008091E8008B7F8093E8008091E8008F7726
:100DD0008093E8000F900F900F900F90CF91DF91CC
:100DE00008950F931F9309EE10E081E0F8018083CE
:100DF00081EC60E06ADA82E0F801808381EC60E0F7
:100E000064DA83E0F801808381E864E35EDA84E0F9
:100E1000F801808380E864E358DA1F910F91089508
:100E2000DF93CF9300D000D0CDB7DEB79091F10023
:100E30002091F100813869F4663009F08FC02132C9
:100E400021F0223209F08AC002C035DF31C046DE0F
:100E50002FC0813209F045C06A3061F16F3F21F047
:100E6000693009F07BC020C0992309F077C02223A4
:100E700009F074C08091F10089838091F1008A8328
:100E800089819A81029709F069C08091E800877F83
:100E90008093E8008091E8008E7F8093E800809145
:100EA000E80080FFFCCF04C0223009F057C0ACDE60
:100EB00081E055C08091F1008B838091F1008C839B
:100EC0008091E800877F8093E8002093090180915A
:100ED000E8008E7F8093E8008091E80080FFFCCFDF
:100EE000E7CF813AD9F5623019F06E3FB9F503C00A
:100EF000892FA8DEDDCF992389F5222379F580910A
:100F0000F10089838091F1008A8389819A81029717
:100F100029F58091E800877F8093E8000E945216AF
:100F200081508093F1008091E8008E7F8093E800EB
:100F30008091E80080FFFCCF8091E80082FFFCCF29
:100F40008091E8008B7F8093E8008091E8008F77A4
:100F50008093E80081E080932A0101C080E00F9037
:100F60000F900F900F90CF91DF91089510922B0169
:100F7000E2EEF0E080818460808310922D0181E0B8
:100F800080932C01089580912B018F5F80932B011A
:100F90000895089510922F0110923001109231019E
:100FA00010923201E4D0482F882329F480910B015C
:100FB000882321F472C08E3109F46FC0642F70E071
:100FC0009B012F7030702A30310531F4809131014E
:100FD00081508093310125C02230310559F4809130
:100FE0003101815080933101809130018F5F809376
:100FF000300120C02330310531F4809130018F5F02
:10100000809330011EC02130310559F480913101A7
:101010008F5F80933101809130018F5F8093300129
:1010200013C02530310531F4809131018F5F8093F9
:10103000310117C02430310521F4809131018F5FD7
:1010400009C02C30310541F02830310551F4809130
:101050003101815080933101809130018150809322
:101060003001CB01807390708031910521F4809123
:101070002F0181600CC08032910521F480912F01F5
:10108000826005C0C09729F480912F01846080930D
:101090002F0140930B0181E0089580E00895809135
:1010A0000C01882309F462C08091D90080FF58C0E8
:1010B00080912601882309F459C080912B01833047
:1010C00008F454C010922B0180912D01882331F433
:1010D00061DF882319F081E080932D0190912D012B
:1010E000992329F480912C01882309F43FC021E041
:1010F0002093E9008091E80085FF38C0992359F0DA
:1011000010922D0110922C0180912F01882369F0FB
:1011100020932C010AC010922F01109230011092DE
:1011200031011092320110922C0180912F01809395
:10113000F100809130018093F10080913101809322
:10114000F100809132018093F1008091E8008E7F60
:101150008093E8008091E8008F778093E8000895FD
:1011600013BE83B7856083BF8895A2CF0895DF93B0
:10117000CF9300D000D0CDB7DEB780B18095898302
:1011800080B180958A8380B180958B8380B1809572
:101190008C8320E0BE016F5F7F4F09C080B1922F2A
:1011A0009370FB01E90FF11D809580832F5F4981CA
:1011B0008A81481799F78B81481781F78C814817E6
:1011C00069F740931201442329F480911101882387
:1011D000F9F452C04E31E1F4809111018E31C1F029
:1011E00080910C01882359F481E080930C0184E6FE
:1011F00090E090930101809300015C9A09C01092E5
:101200000C0182E390E090930101809300015C98CF
:1012100090911101842F8923891769F01092100190
:1012200010920F014093110180910201882381F0F7
:101230001092020122C0892F842B891759F081E076
:10124000809302011092100110920F01409311013E
:1012500090E013C020910F013091100180910001A6
:10126000909101012817390738F42F5F3F4F3093D1
:10127000100120930F01ECCF942F892F0F900F9026
:101280000F900F90CF91DF91089511B88FEF82B931
:101290008AB1806F8AB910922E01E2EEF0E080816F
:1012A000846080830895982F882361F480910D01D4
:1012B000803EE8F58823D9F110920D0110920E01BD
:1012C00020E045C0833EF1F0843E38F4813E91F049
:1012D000823EA0F4803E59F509C0853ED9F0853E96
:1012E000A8F0863ED9F0873E11F51CC080910E0112
:1012F00081601BC080910E01826017C080910E0139
:10130000846013C080910E0188600FC080910E012F
:1013100080610BC080910E01806207C080910E0138
:10132000806403C080910E01806880930E0120913B
:101330000E01222311F05D9A01C05D98993329F4C2
:1013400080910D01893309F04E9A90930D01822FFF
:10135000089580910C01882309F03FC082E08093BA
:10136000E9008091E80080FF38C080912601882341
:10137000A1F18091E80080FFFCCFF9DE8093340179
:10138000863510F010923401E0913401F0E0E3541E
:10139000FE4FE491E093340182E08093E9008E2FC8
:1013A00082DF8093F1001092F100809134018093EC
:1013B000F1001092F1001092F1001092F1001092E1
:1013C000F1001092F1008091E8008E7F8093E80098
:1013D0008091E8008F778093E80008951F9383E061
:1013E0008093E90013E009C01092E9008091E800C1
:1013F00083FF01C029D81093E9008091EB0085FD9F
:10140000F3CF84E08093E90014E009C01092E90072
:101410008091E80083FF01C017D81093E900809104
:10142000EB0085FDF3CF83E08093E90004C0809159
:10143000EB0080FF38C08091E80085FFF8CF85E59C
:101440008093F10093E59093F10082E48093F100A2
:101450009093F100809113018093F1008091140129
:101460008093F100809115018093F1008091160125
:101470008093F100809137018093F10080913801D1
:101480008093F100809139018093F10080913A01BD
:101490008093F10080914B018093F1008091E800EE
:1014A0008F778093E8001F91089584E08093E9008E
:1014B0002091F1008091F100833519F490E02535F9
:1014C00009F091E08091F100823409F091E080917F
:1014D000F100833411F49923B1F08091E8008B7FFF
:1014E0008093E8008091E8008F778093E80083E0A4
:1014F0008093E9008091EB0080628093EB0081E0B3
:101500008093220108958091F100809313018091CE
:10151000F100809314018091F10080931501809176
:10152000F100809316018091F10080933701809142
:10153000F100809338018091F1008093390180910E
:10154000F10080933A018091F100882321F081E03D
:101550008093360102C0109236018091F100809391
:10156000350180912A01882321F40E94541680932A
:1015700035018091F100EBE3F1E08091F10081937E
:1015800081E0EB34F807C9F78091E8008B7F809306
:10159000E8008091E8008F778093E8008091360121
:1015A000813019F483E08093E9000E9409168130AC
:1015B00089F08091EB0080628093EB00809136018E
:1015C000813011F0E4E001C0E3E0F0E0E15EFE4FC5
:1015D00081E08083089580912601882349F084E08A
:1015E0008093E9008091E80082FF02C05EDFF6CEC2
:1015F00008958AB1806F8AB9E2EEF0E0808184605C
:10160000808394C0809117010895BF92CF92DF929A
:10161000EF92FF920F931F93DF93CF9300D000D0F0
:10162000CDB7DEB769837A838B839C836A01BB2441
:10163000B39440C0E980FA800B811C81C801B701D6
:1016400066D1898180FD25C081E0C816D10479F476
:1016500081E090E0F7D1B82EF1D10894E11CF11CA3
:10166000011D111DE982FA820B831C832AC082E0CE
:1016700090E0E8D1B82EE2D1AEEFBFEFCA0EDB1E8C
:1016800082E090E0A0E0B0E0E80EF91E0A1F1B1F08
:101690000DC081E090E0D6D1B82ED0D10894C10819
:1016A000D1080894E11CF11C011D111DE982FA8288
:1016B0000B831C83C114D10421F091E0B91609F405
:1016C000B9CFBCD120E030E0BB2011F421E030E004
:1016D000C9010F900F900F900F90CF91DF911F9144
:1016E0000F91FF90EF90DF90CF90BF900895909171
:1016F000170180911801981729F09093180123E0A1
:1017000030E008C0B2D0813019F022E030E002C0F1
:1017100020E030E0C9010895FC018FEF9FE7A0E0D1
:10172000B0E080839183A283B383E1CF75C0089535
:10173000CF92DF92EF92FF920F931F93DF93CF939D
:1017400000D000D0CDB7DEB78B019C01809117018E
:101750008823D1F409831A832B833C836A0147C011
:10176000E980FA800B811C81C801B70164D38981AB
:1017700080FD2BC081E0C816D104A1F481E090E087
:101780003CD4882321F448D021E030E037C002D493
:101790000894E11CF11C011D111DE982FA820B83E2
:1017A0001C8329C082E090E028D4882361F3F2D31F
:1017B000AEEFBFEFCA0EDB1E82E090E0A0E0B0E02B
:1017C000E80EF91E0A1F1B1F0EC081E090E015D421
:1017D0008823C9F2DFD30894C108D1080894E11C1A
:1017E000F11C011D111DE982FA820B831C83C114B7
:1017F000D10409F0B5CFCED320E030E0C9010F907D
:101800000F900F900F90CF91DF911F910F91FF904C
:10181000EF90DF90CF900895239884B1876084B9CA
:1018200085B18F6085B98DB183608DB98EB18360CC
:101830008EB98CB580618CBD8CB5837F8CBD8CB529
:101840008C608CBD84B1866084B98CB58C7F8CBD76
:101850008CB58CBD8DB581608DBD8CB580648CBD23
:1018600010921D0110921E01089510921E0190E029
:1018700037ED24C08EB183608EB9992319F0913071
:1018800021F402C0709801C071983EBD0DB407FEEE
:10189000FDCF1EBC0DB407FEFDCF8EB5292F2F5FE7
:1018A0008C738C3339F090931E018EB183608EB9A6
:1018B00080E008958EB183608EB9922F9230D0F27D
:1018C00090931E0181E008958EB183608EB980915E
:1018D0001E01882319F0813021F402C0709801C0E4
:1018E000719887ED8EBD0DB407FEFDCF1EBC0DB403
:1018F00007FEFDCF04C01EBC0DB407FEFDCF0EB425
:1019000007FEF9CF8EB183608EB98EB508951F930F
:10191000DF93CF9300D000D0CDB7DEB7AC01162F48
:1019200069837A838B839C83CB01DA019C01AD01AF
:10193000217030704070507079E0220F331F441FC7
:10194000551F7A95D1F78C7FBA2FA92F982F88270A
:10195000282B392B4A2B5B2B2093190130931A012A
:1019600040931B0150931C011695117010931E019A
:1019700020911D01822F90E0012E02C09595879540
:101980000A94E2F780FF0DC081E090E0012E02C0D2
:10199000880F991F0A94E2F78095822380931D0196
:1019A00093DF8EB183608EB9112319F0113021F4C9
:1019B00002C0709801C0719882ED8EBD0DB407FE13
:1019C000FDCF20911A0180911B01880F922F991F42
:1019D0009927991F892B8EBD0DB407FEFDCF822F4D
:1019E00090E08C7F880F991F2370282B2EBD0DB49B
:1019F00007FEFDCF809119018EBD0DB407FEFDCF0E
:101A00008FEF8EBD0DB407FEFDCF8FEF8EBD0DB4F1
:101A100007FEFDCF8FEF8EBD0DB407FEFDCF8FEF1C
:101A20008EBD0DB407FEFDCF8EB581E00F900F90F7
:101A30000F900F90CF91DF911F9108958EB1836029
:101A40008EB90895BC012091190130911A0140917D
:101A50001B0150911C0198E0F8941EBC0DB407FEC8
:101A6000FDCF8EB58093F1001EBC0DB407FEFDCFF7
:101A70008EB58093F1001EBC0DB407FEFDCF8EB570
:101A80008093F1001EBC0DB407FEFDCF8EB5809390
:101A9000F1001EBC0DB407FEFDCF8EB58093F100A2
:101AA0001EBC0DB407FEFDCF8EB58093F1001EBCA9
:101AB0000DB407FEFDCF8EB58093F1001EBC0DB4B2
:101AC00007FEFDCF8EB58093F1001EBC0DB407FE5E
:101AD000FDCF8EB58093F1001EBC0DB407FEFDCF87
:101AE0008EB58093F1001EBC0DB407FEFDCF8EB500
:101AF0008093F1001EBC0DB407FEFDCF8EB5809320
:101B0000F1001EBC0DB407FEFDCF8EB58093F10031
:101B10001EBC0DB407FEFDCF8EB58093F1001EBC38
:101B20000DB407FEFDCF8EB58093F1001EBC0DB441
:101B300007FEFDCF8EB58093F1001EBC0DB407FEED
:101B4000FDCF8EB58093F1001EBC0DB407FEFDCF16
:101B50008EB58093F1001EBC0DB407FEFDCF8EB58F
:101B60008093F1001EBC0DB407FEFDCF8EB58093AF
:101B7000F1001EBC0DB407FEFDCF8EB58093F100C1
:101B80001EBC0DB407FEFDCF8EB58093F1001EBCC8
:101B90000DB407FEFDCF8EB58093F1001EBC0DB4D1
:101BA00007FEFDCF8EB58093F1001EBC0DB407FE7D
:101BB000FDCF8EB58093F1001EBC0DB407FEFDCFA6
:101BC0008EB58093F1001EBC0DB407FEFDCF8EB51F
:101BD0008093F1001EBC0DB407FEFDCF8EB580933F
:101BE000F1001EBC0DB407FEFDCF8EB58093F10051
:101BF0001EBC0DB407FEFDCF8EB58093F1001EBC58
:101C00000DB407FEFDCF8EB58093F1001EBC0DB460
:101C100007FEFDCF8EB58093F1001EBC0DB407FE0C
:101C2000FDCF8EB58093F1001EBC0DB407FEFDCF35
:101C30008EB58093F1001EBC0DB407FEFDCF8EB5AE
:101C40008093F1001EBC0DB407FEFDCF8EB58093CE
:101C5000F1001EBC0DB407FEFDCF8EB58093F100E0
:101C60001EBC0DB407FEFDCF8EB58093F1001EBCE7
:101C70000DB407FEFDCF8EB58093F1001EBC0DB4F0
:101C800007FEFDCF8EB58093F1001EBC0DB407FE9C
:101C9000FDCF8EB58093F1001EBC0DB407FEFDCFC5
:101CA0008EB58093F1001EBC0DB407FEFDCF8EB53E
:101CB0008093F1001EBC0DB407FEFDCF8EB580935E
:101CC000F1001EBC0DB407FEFDCF8EB58093F10070
:101CD0001EBC0DB407FEFDCF8EB58093F1001EBC77
:101CE0000DB407FEFDCF8EB58093F1001EBC0DB480
:101CF00007FEFDCF8EB58093F1001EBC0DB407FE2C
:101D0000FDCF8EB58093F1001EBC0DB407FEFDCF54
:101D10008EB58093F1001EBC0DB407FEFDCF8EB5CD
:101D20008093F1001EBC0DB407FEFDCF8EB58093ED
:101D3000F1001EBC0DB407FEFDCF8EB58093F100FF
:101D40001EBC0DB407FEFDCF8EB58093F1001EBC06
:101D50000DB407FEFDCF8EB58093F1001EBC0DB40F
:101D600007FEFDCF8EB58093F1001EBC0DB407FEBB
:101D7000FDCF8EB58093F1001EBC0DB407FEFDCFE4
:101D80008EB58093F1001EBC0DB407FEFDCF8EB55D
:101D90008093F1001EBC0DB407FEFDCF8EB580937D
:101DA000F1001EBC0DB407FEFDCF8EB58093F1008F
:101DB0001EBC0DB407FEFDCF8EB58093F1001EBC96
:101DC0000DB407FEFDCF8EB58093F1001EBC0DB49F
:101DD00007FEFDCF8EB58093F1008091E8008F77EC
:101DE0008093E800789404C08091EB0080FF19C0D4
:101DF0008091E80085FFF8CF915009F02DCE20505A
:101E00003E4F4F4F5F4F6150704009F024CE2093FA
:101E1000190130931A0140931B0150931C0181E07A
:101E200008952093190130931A0140931B01509398
:101E30001C0180E008951F93DF93CF9300D000D062
:101E4000CDB7DEB7AC01162F69837A838B839C8371
:101E5000CB01DA019C01AD012170307040705070EF
:101E600069E0220F331F441F551F6A95D1F78C7FFD
:101E7000BA2FA92F982F8827282B392B4A2B5B2B79
:101E80002093190130931A0140931B0150931C01B8
:101E90001695117010931E0120911D01822F90E064
:101EA000012E02C0959587950A94E2F780FF0DC038
:101EB00081E090E0012E02C0880F991F0A94E2F79A
:101EC0008095822380931D01FFDC8EB183608EB9E3
:101ED000112319F0113021F402C0709801C07198DB
:101EE00083E58EBD0DB407FEFDCF20911A018091D0
:101EF0001B01880F922F991F9927991F892B8EBD3F
:101F00000DB407FEFDCF220F2EBD0DB407FEFDCF91
:101F10001EBC0DB407FEFDCF8EB58EB183608EB9A9
:101F2000D3DC8EB183608EB9112319F0113021F406
:101F300002C0709801C0719882E88EBD0DB407FE92
:101F4000FDCF20911A0180911B01880F922F991FBC
:101F50009927991F892B8EBD0DB407FEFDCF822FC7
:101F600090E08C7F880F991F2370282B2EBD0DB415
:101F700007FEFDCF809119018EBD0DB407FEFDCF88
:101F80008EB581E00F900F900F900F90CF91DF9161
:101F90001F91089517C01EBC0DB407FEFDCF8091A0
:101FA000190190911A01A0911B01B0911C01019699
:101FB000A11DB11D8093190190931A01A0931B01DB
:101FC000B0931C0180911901882329F780911A018F
:101FD00080FDE1CF8EB58EB183608EB981E090E057
:101FE00000901E0102C0880F991F0A94E2F7209109
:101FF0001D01282B20931D0108959C0181E090E094
:1020000000901E0102C0880F991F0A94E2F7582F12
:1020100040911D0198E004C08091EB0080FFBDC19C
:102020008091E80085FFF8CFF8948091F1008EBD93
:102030000DB407FEFDCF8091F1008EBD0DB407FEFB
:10204000FDCF8091F1008EBD0DB407FEFDCF8091D4
:10205000F1008EBD0DB407FEFDCF8091F1008EBD65
:102060000DB407FEFDCF8091F1008EBD0DB407FECB
:10207000FDCF8091F1008EBD0DB407FEFDCF8091A4
:10208000F1008EBD0DB407FEFDCF8091F1008EBD35
:102090000DB407FEFDCF8091F1008EBD0DB407FE9B
:1020A000FDCF8091F1008EBD0DB407FEFDCF809174
:1020B000F1008EBD0DB407FEFDCF8091F1008EBD05
:1020C0000DB407FEFDCF8091F1008EBD0DB407FE6B
:1020D000FDCF8091F1008EBD0DB407FEFDCF809144
:1020E000F1008EBD0DB407FEFDCF8091F1008EBDD5
:1020F0000DB407FEFDCF8091F1008EBD0DB407FE3B
:10210000FDCF8091F1008EBD0DB407FEFDCF809113
:10211000F1008EBD0DB407FEFDCF8091F1008EBDA4
:102120000DB407FEFDCF8091F1008EBD0DB407FE0A
:10213000FDCF8091F1008EBD0DB407FEFDCF8091E3
:10214000F1008EBD0DB407FEFDCF8091F1008EBD74
:102150000DB407FEFDCF8091F1008EBD0DB407FEDA
:10216000FDCF8091F1008EBD0DB407FEFDCF8091B3
:10217000F1008EBD0DB407FEFDCF8091F1008EBD44
:102180000DB407FEFDCF8091F1008EBD0DB407FEAA
:10219000FDCF8091F1008EBD0DB407FEFDCF809183
:1021A000F1008EBD0DB407FEFDCF8091F1008EBD14
:1021B0000DB407FEFDCF8091F1008EBD0DB407FE7A
:1021C000FDCF8091F1008EBD0DB407FEFDCF809153
:1021D000F1008EBD0DB407FEFDCF8091F1008EBDE4
:1021E0000DB407FEFDCF8091F1008EBD0DB407FE4A
:1021F000FDCF8091F1008EBD0DB407FEFDCF809123
:10220000F1008EBD0DB407FEFDCF8091F1008EBDB3
:102210000DB407FEFDCF8091F1008EBD0DB407FE19
:10222000FDCF8091F1008EBD0DB407FEFDCF8091F2
:10223000F1008EBD0DB407FEFDCF8091F1008EBD83
:102240000DB407FEFDCF8091F1008EBD0DB407FEE9
:10225000FDCF8091F1008EBD0DB407FEFDCF8091C2
:10226000F1008EBD0DB407FEFDCF8091F1008EBD53
:102270000DB407FEFDCF8091F1008EBD0DB407FEB9
:10228000FDCF8091F1008EBD0DB407FEFDCF809192
:10229000F1008EBD0DB407FEFDCF8091F1008EBD23
:1022A0000DB407FEFDCF8091F1008EBD0DB407FE89
:1022B000FDCF8091F1008EBD0DB407FEFDCF809162
:1022C000F1008EBD0DB407FEFDCF8091F1008EBDF3
:1022D0000DB407FEFDCF8091F1008EBD0DB407FE59
:1022E000FDCF8091F1008EBD0DB407FEFDCF809132
:1022F000F1008EBD0DB407FEFDCF8091F1008EBDC3
:102300000DB407FEFDCF8091F1008EBD0DB407FE28
:10231000FDCF8091F1008EBD0DB407FEFDCF809101
:10232000F1008EBD0DB407FEFDCF8EB58091E800A3
:102330008B7F8093E8008091E8008F778093E8009E
:102340007894915009F06CCE8091190190911A0106
:10235000A0911B01B0911C0180509E4FAF4FBF4F09
:102360008093190190931A01A0931B01B0931C0153
:102370002150304080911A0190E083709070892B39
:1023800021F48EB183608EB9452B2115310509F0FA
:1023900041CE40931D0181E0089540931D0180E0EE
:1023A0000895DF93CF93CDB7DEB762970FB6F89459
:1023B000DEBF0FBECDBF40913F01433108F042E187
:1023C00080E789831A8280914C018B831C821D8255
:1023D0001E821F828AE0888719861A861B861C86C1
:1023E00080914D018D8780914E018E871F86188ABE
:1023F000198A1A8A9E012F5F3F4FF90103C081910C
:102400008093F1008E2F821B8417C8F38091E8001F
:102410008F778093E8008091370190913801A091E7
:102420003901B0913A01841B9109A109B109809346
:10243000370190933801A0933901B0933A0110927B
:102440004B0110924C0110924D0110924E0181E00F
:1024500062960FB6F894DEBF0FBECDBFCF91DF916D
:10246000089580913C0190E083709070892B21F455
:1024700080913D01882369F081E080934B0185E0E4
:1024800080934C0184E280934D0110924E0180E0D4
:10249000089590913F01913608F090E620E0EFE238
:1024A000F2E015C0283019F4E3E1F2E009C0203170
:1024B00019F4EBE1F2E004C0203211F4EBE2F2E0B7
:1024C00084918093F1002F5F243219F031962917FF
:1024D00048F38091E8008F778093E800809137017E
:1024E00090913801A0913901B0913A01821B910974
:1024F000A109B1098093370190933801A093390164
:10250000B0933A0110924B0110924C0110924D0180
:1025100010924E0181E008951F93182F882311F027
:102520001092F1006093F1001092F100809135015A
:10253000D7D3882321F080E88093F10002C0109265
:10254000F100112331F01092F1001092F10010927D
:10255000F1001092F1001F9108951F93282F8823F6
:1025600019F01091430102C010913F0180913D018B
:1025700090E08F7390708C31910541F08F3391050D
:1025800009F456C0019709F0F1C020C0822F6FE016
:10259000C3DF8CE18093F1008AE08093F100109218
:1025A000F10085E08093F1001092F1001092F100AB
:1025B0001092F1001092F1001092F1001092F100CF
:1025C0001092F10081E08093F10021C0822F6FE032
:1025D000A3DF81E08093F1008AE08093F10090E82E
:1025E0009093F10083E08093F1001092F10010923B
:1025F000F1001092F1001092F1001D3040F0909324
:10260000F1001092F1001092F1001092F10080910F
:10261000E8008F778093E80080913701909138012E
:10262000A0913901B0913A014097A109B10939C08F
:10263000222359F01D3110F06BE102C0612F62506E
:10264000822F6ADF1830B1F50BC01C3110F06BE13E
:1026500002C0612F615080E05FDF143059F511C076
:102660008091E8008F778093E80080913701909106
:102670003801A0913901B0913A010897A109B10937
:1026800010C08091E8008F778093E8008091370137
:1026900090913801A0913901B0913A010497A109B4
:1026A000B1098093370190933801A0933901B09319
:1026B0003A0169C071E07093F1006AE06093F10043
:1026C00090E89093F10083E08093F1001092F10084
:1026D0001092F1001092F1001092F1002091370158
:1026E000309138014091390150913A011D3060F12B
:1026F0009093F1001092F1001092F1001092F1000D
:102700008CE18093F1006093F1001092F10085E07C
:102710008093F1001092F1001092F1001092F100FC
:102720001092F1001092F1001092F1001092F1005D
:102730007093F1008091E8008F778093E8002C512E
:1027400030404040504009C08091E8008F7780932E
:10275000E800211B310941095109209337013093C9
:1027600038014093390150933A010DC081E08093C4
:102770004B0185E080934C0184E280934D011092DF
:102780004E0180E009C010924B0110924C01109252
:102790004D0110924E0181E01F9108950F931F93F8
:1027A000DF93CF9300D000D000D0CDB7DEB7FE01CD
:1027B000339680913D01838380913E018283809195
:1027C0003F018183809140018B83809142018A8304
:1027D00080914301898380913601813039F480935F
:1027E0004B0185E080934C0184E292C080913701D7
:1027F00090913801A0913901B0913A010097A1055B
:10280000B105C1F489819A81892B39F410924B0169
:1028100010924C0110924D0109C081E080934B0150
:1028200085E080934C0184E280934D0110924E012B
:1028300081E07CC08091350153D2813039F480939E
:102840004B0187E080934C0187E262C04B815C8141
:102850006D817E81009137011091380120913901FD
:1028600030913A01E9E03695279517950795EA9555
:10287000D1F780913501980119D282309105C9F1C3
:1028800083309105F1F1892B09F045C029813A8106
:1028900040E050E08091370190913801A0913901DA
:1028A000B0913A0169E0B695A795979587956A9595
:1028B000D1F7281739074A075B0739F410924B0103
:1028C00010924C0110924D0109C081E080934B01A0
:1028D00085E080934C0184E280934D0110924E017B
:1028E00010923701109238011092390110923A017A
:1028F0009FCF81E080934B0182E080934C018AE37B
:1029000007C081E080934B0186E080934C0188E210
:1029100080934D0108C081E080934B0184E0809357
:102920004C0110924D0110924E0180E026960FB698
:10293000F894DEBF0FBECDBFCF91DF911F910F91F5
:1029400008950F931F93DF93CF9300D000D000D052
:10295000CDB7DEB7FE01339680913D018383809130
:102960003E01828380913F018183809140018B836E
:10297000809142018A83809143018983809136014D
:10298000882341F481E080934B0185E080934C01E2
:1029900084E280C000913701109138012091390103
:1029A00030913A010115110521053105B9F48981EC
:1029B0009A81892B39F410924B0110924C0110929C
:1029C0004D0109C081E080934B0185E080934C016B
:1029D00084E280934D0110924E014BC04B815C818B
:1029E0006D817E81A9E03695279517950795AA9563
:1029F000D1F780913501980166D182309105D9F1E6
:102A00008330910509F43FC0892B09F046C0298124
:102A10003A8140E050E08091370190913801A091D7
:102A20003901B0913A01F9E0B695A7959795879548
:102A3000FA95D1F7281739074A075B0739F410923E
:102A40004B0110924C0110924D0109C081E080931E
:102A50004B0185E080934C0184E280934D011092FC
:102A60004E011092370110923801109239011092E4
:102A70003A0181E01DC081E080934B0182E08093A8
:102A80004C018AE307C081E080934B0186E080938C
:102A90004C0188E280934D0108C081E080934B0196
:102AA00084E080934C0110924D0110924E0180E021
:102AB00026960FB6F894DEBF0FBECDBFCF91DF9143
:102AC0001F910F9108950F931F93DF93CF9300D021
:102AD00000D0CDB7DEB7809135018E010F5F1F4F5B
:102AE000B80104D18230910509F43FC083309105CB
:102AF00009F443C0892B09F04AC0F801838180930F
:102B0000F10082818093F10081818093F1008081C6
:102B10008093F1001092F1001092F10082E0809316
:102B2000F1001092F1008091E8008F778093E80027
:102B30008091370190913801A0913901B0913A010B
:102B40000897A109B1098093370190933801A093A8
:102B50003901B0933A0110924B0110924C0110923E
:102B60004D0110924E0181E01DC081E080934B0128
:102B700082E080934C018AE307C081E080934B019F
:102B800086E080934C0188E280934D0108C081E08B
:102B900080934B0184E080934C0110924D01109280
:102BA0004E0180E00F900F900F900F90CF91DF912A
:102BB0001F910F91089580913501A3D08230910526
:102BC00051F08330910579F0892BB9F410924B01C3
:102BD00010924C0118C081E080934B0182E08093F9
:102BE0004C018AE307C081E080934B0186E080932B
:102BF0004C0188E280934D0108C081E080934B0135
:102C000084E080934C0110924D0110924E0181E0BE
:102C1000089580913B018A3221F45F9ABFDD5F986D
:102C20000895883221F45D9A8CDE5D9808958B3189
:102C300011F18C3160F48330B1F0843018F48823C2
:102C4000A1F023C0823181F08A31F9F410C08532BD
:102C500069F0863218F48E31C1F40DC08F3259F00C
:102C60008A3599F406C09DCBFCCBA5CF2CCF80E054
:102C700001C081E072CC10924B0110924C01109275
:102C80004D0110924E0181E0089581E080934B0147
:102C900085E080934C0180E280934D0110924E01BB
:102CA00080E0089581E0089580E00895882319F078
:102CB00021E030E006C0CB01BA01A9010E94980BC7
:102CC0009C01C9010895882319F021E030E006C075
:102CD000CB01BA01A9010E94050B9C01C90108950D
:102CE000882311F081E008950C94020B882319F0D9
:102CF00021E030E004C0CB010E948C0B9C01C90193
:102D00000895882319F021E030E003C00E94770B7A
:102D10009C01C90108950E94470180E090E020E8ED
:102D20000FB6F89420936100809361000FBE0E945B
:0C2D3000630180E090E00895F894FFCF6C
:042D3C003200010060
:00000001FF
